:100000000C94ED020C9431030C9431030C943103E5
:100010000C9431030C9431030C9431030C94310390
:100020000C9431030C9431030C94C10F0C94931075
:100030000C9431030C9431030C9431030C94310370
:100040000C9431030C94FD220C9431030C94310375
:100050000C9431030C94DF1D0C9431030C94310388
:100060000C9431030C9431030C9431030C94310340
:100070000C9431030C9431030C9431030C94310330
:100080000C9431030C9431030C9431030C94310320
:100090000C9431030C9431030C9431030C94310310
:1000A0000C9431030C9431030C943103AB05DF0540
:1000B00004064206AB05E8052606500605070507B7
:1000C000D406DC06E406F2060011221110122211F9
:1000D000101267118A111012DF11F211C114C1142C
:1000E000F014F01426154615771677165115771665
:1000F0000116011668167716771671160E160E166B
:100100000E160E160E160E160E160E160E160E16CF
:100110000E160E160E160E160E160E1620162D168E
:1001200034163B16451600000000000000000000D9
:10013000000000000000000000000AC80BC80CC846
:100140000DC80EC80FC810C811C80D200C200B30E8
:100150000A30E00000001E00140004001D0000072B
:100160004E001F001A0016001B00000F4C0020005C
:10017000080007000600E2002A002100150009001F
:100180001900E3004B00220017000A0005000000E0
:100190004A0029002F0000002B0200004D002D0016
:1001A000300000002B000000500023001C000B005A
:1001B000110000004F00240018000D001000E7009F
:1001C000520025000C000E003600E6002C00260030
:1001D00012000F003700000F280027001300330023
:1001E000380000075100112010200F200E30E400CD
:1001F00000000100010001000100E00000003A00E1
:100200001E0220022202000751003B001F022102B1
:100210002302000F28003C002F0226022F00E200DC
:100220002C003D00300227023000E30052003E0067
:10023000240235003502000050002900360200007B
:100240002B0000004F002D00370200002B020000A1
:100250004A003F0031023800310000004D004000EC
:10026000240021001E0027684B00410025002200C9
:100270001F0037644C0042002600230020002E6F30
:100280002A004300380025022D002E674E00010091
:1002900001000100010028610000010001000100CF
:1002A0000100E000000044006600A6000000000716
:1002B000B50045001430F2001630F600000068006A
:1002C000F000F100F100F400B60069001530F30011
:1002D0001730F500B4006A00A900AA00A8000000C9
:1002E000B8002900F9000000FA000000B900000081
:1002F000F9000000FA000000AC006B00460053005B
:1003000000000000AB006C004A0050004D0049683E
:10031000A9006D005200510051004C64AE006E0007
:100320004B004F004E00000FAD006F00B100B30056
:1003300000000007AA000100010001000100E40024
:10034000000001000100010001000100000029007F
:100350000100010001000100010001000100010095
:100360000100010001000100010001000100010085
:100370000100010001000100010001000100010075
:100380000100010001000000010001000100000067
:100390000100000001000100010000000100000058
:1003A0000100010001000100010000000100010046
:1003B0000100010001000100010001000100010035
:1003C0000100010001000100010001000100010025
:1003D00001002A00010001000100010001000100EC
:1003E00001000100E5000100000016034500720055
:1003F00067006F0044006F007800200045005A003D
:10040000000016034500720067006F0044006F0093
:100410007800200045005A00000004030904090286
:100420006D00040100A0FA090400000103010100AD
:100430000921110100012240000705810308000A7B
:100440000904010001030102000921110100012238
:100450004D000705820308000A0904020001030099
:10046000000009211101000122360007058303085D
:10047000000A090403000103000000092111010022
:100480000122390007058403100001120110010048
:10049000000008EDFE07130100010200010501093B
:1004A00006A101050719E029E71500250195087542
:1004B000018102050819012905950575019102952B
:1004C000017503910105071900297715002501958C
:1004D0007875018102C005010980A101850216011C
:1004E0000026B7001A01002AB70075109501810097
:1004F000C0050C0901A1018503160100269C021A02
:1005000001002A9C02751095018100C005010902B5
:10051000A1010901A10005091901290515002501FD
:100520009505750181029501750381010501093069
:1005300009311581257F95027508810609381581D5
:10054000257F950175088106050C0A38021581255D
:100550007F950175088106C0C005010906A1010546
:100560000719E029E7150025019508750181029515
:100570000175088101050819012905950575019185
:10058000029501750391010507190029FF15002641
:10059000FF00950675088100C00000000000000003
:1005A00000000000010204060A0F17202C3A4A5DE1
:1005B00071879DB3C7DAE9F5FCFFFCF5E9DAC7B34B
:1005C0009D87715D4A3A2C20170F0A06040201002C
:1005D0000000000000000000000011241FBECFEF4B
:1005E000DAE0DEBFCDBF04B603FE24C08091050271
:1005F00090910602A0910702B09108028730904BBB
:10060000A740B04BB9F41092050210920602109266
:1006100007021092080214BE84B7877F84BF88E166
:100620000FB6F89480936000109260000FBEE0E077
:10063000FFE3099511E0A0E0B1E0E8E8F9E402C0C9
:1006400005900D92A433B107D9F712E0A4E3B1E00D
:1006500001C01D92A530B107E1F70E94090D0C946D
:10066000C2240C9400001092B9008AE08093B80074
:10067000089594EA9093BC009091BC0097FFFCCF42
:100680009091B900987F983021F0903111F081E07D
:1006900008958093BB0084E88093BC008091BC00E7
:1006A00087FFFCCF8091B900887F883111F08034BA
:1006B00071F780E0089584E98093BC008091BC00CC
:1006C00084FDFCCF08958093BB0084E88093BC0038
:1006D0008091BC0087FFFCCF9091B900987F81E0AA
:1006E000983209F480E0089584E88093BC008091FA
:1006F000BC0087FFFCCF8091BB00089580B38C7055
:1007000080BB81B3836F81BB08958091010181110A
:1007100015C080E40E9439038093010181110CC04F
:1007200082E10E94630380930101811105C08FEF74
:100730000E946303809301010E945B0384B1807F68
:1007400084B985B1807F85B98AB1837F8AB98BB13D
:10075000837F8BB93E98469808950E944F058093F9
:1007600001010E9485030E947E03A5E3B1E0E3E45A
:10077000F1E08EE08E0F11921D928E13FCCF0C943F
:1007800039050E944F05809301010E9485030E9454
:100790007E03A5E3B1E0E3E4F1E08EE08E0F119279
:1007A0001D928E13FCCF0895BF92CF92DF92EF92ED
:1007B000FF920F931F93CF93DF93809101018823C2
:1007C00079F0809134018F5F80933401811108C0EA
:1007D0000E944F0580930101811102C00E94E10433
:1007E00005E311E0C0E0D0E0DD24D39482E0C82E20
:1007F000EE24E394F12CC730D10500F5809101017E
:10080000811164C080E40E94390380930101811149
:1008100012C082E10E9463038093010181110BC029
:10082000C7010C2E01C0880F0A94EAF780950E9438
:100830006303809301010E945B0348C0CA30A1F0AA
:1008400028F4C83059F0C93061F005C0CC3089F0C7
:1008500070F0CD3089F0209A289810C0219A2998FC
:100860000DC0229A2A980AC0239A2B9807C0529A40
:1008700001C0539A5B9802C03E9A469890EA9A95B6
:10088000F1F79FB1799902C082E001C080E09170D8
:100890009D25982B7C9902C084E001C080E0892BC3
:1008A0007D9902C038E001C030E0832B7E9902C000
:1008B00020E101C020E0822B9FB19095991F9927DC
:1008C000991F9295990F907E892B0FC080910101FD
:1008D000811149C080E40E9439038093010188237B
:1008E00079F1B12C0E945B038B2DF8019081981750
:1008F00019F08083C09200010E94850321960F5F4A
:100900001F4FCE30D10509F076CF809100018823AA
:1009100061F1815080930001882339F08FE99FE0D5
:100920000197F1F700C0000020C0A3E4B1E0E5E3C7
:10093000F1E0CF01825F91919D938E13FCCF15C0A2
:1009400083E10E946303809301018111CACF81E496
:100950000E943903809301018111C3CF0E94740367
:10096000B82EB094BFCF80E0C0CF0E94DF0481E0FA
:10097000DF91CF911F910F91FF90EF90DF90CF907B
:10098000BF900895E82FF0E0ED5BFE4F8081089561
:1009900008950F931F93CF93DF93C3E4D1E010E04A
:1009A0000C2F025F899190E00E94561D180F0C13C6
:1009B000F9CF812FDF91CF911F910F9108950C9462
:1009C000090756985E9825982D9826982E9827986E
:1009D0002F988FEF90E090938900809388009093F8
:1009E0008B0080938A0090938D0080938C00259AD1
:1009F0002D9A2FEF80E792E0215080409040E1F760
:100A000000C00000269A2E9A2FEF80E792E0215036
:100A100080409040E1F700C00000279A2F9A2FEF06
:100A200080E792E0215080409040E1F700C0000054
:100A300025982D982FEF80E792E02150804090403C
:100A4000E1F700C0000026982E982FEF80E792E093
:100A5000215080409040E1F700C0000027982F9877
:100A600056985E9825982D9826982E9827982F9816
:100A7000089589EA8093800089E08093810024981A
:100A80002C983F988AB18F748AB96E98479A8BB127
:100A9000806B8BB9769A0E94E1040C94080780E27F
:100AA000809301018091510181110EC00E94330396
:100AB00081E0809351012FEF83ED90E3215080403E
:100AC0009040E1F700C0000080E40E943903809369
:100AD000010181112EC00E946303809301018111E5
:100AE00028C00E94630380930101811122C08FE31B
:100AF0000E9463038093010181111BC00E945B036C
:100B000080E40E94390380930101811112C08CE0BE
:100B10000E9463038093010181110BC00E94630353
:100B200080930101811105C08FE30E9463038093CC
:100B300001010E945B03809101010895462F50E05E
:100B4000FA013A97EE30F10508F05FC1DC01EA5A8C
:100B5000FF4F0C94722412962C9112978091580199
:100B6000909159012223F9F015962C91207FD9F408
:100B700001968330910510F082E090E09093590146
:100B800080935801809158019091590182309105CC
:100B900029F489E30E94651389E30EC0019709F0E7
:100BA00034C181EEFAC001979093590180935801A6
:100BB000892B09F02AC181EE0E942D1426C11296BC
:100BC0002C918091560190915701222379F090C089
:100BD00012963C91129715962C9180915601909106
:100BE0005701207F31117AC009F09FC0019790937F
:100BF000570180935601892B09F007C18091530159
:100C0000811103C181E067C012963C91129715963D
:100C10002C918091540190915501207F332361F0F4
:100C2000222309F491C0009709F08EC0209152014F
:100C300021118AC08BE2B1C02223B1F00097A1F448
:100C400020915201211110C08BE2B6CF12963C9137
:100C5000129715962C918091540190915501207F07
:100C6000311168C009F08DC00197909355018093B0
:100C70005401892B09F0C9C0809152018111C5C06E
:100C800082E029C012969C91129715968C91992317
:100C9000B1F0982F907F79F080FD0DC085E37DC085
:100CA00012969C91129715968C91992379F0982F12
:100CB000907F09F06FC083E00E941F1BA6C0982F91
:100CC000907F41F080FD06C085E376CF982F907F1E
:100CD00009F066C083E00E94401B97C0222341F0C8
:100CE000009731F420915301211102C084E355C0D3
:100CF00001968330910510F082E090E090935701C7
:100D00008093560180915601909157018230910550
:100D100029F0019709F079C081E0CECF909153017D
:100D200081E089278093530170C0009709F05ECF5E
:100D300084E342CF222341F0009731F42091520105
:100D4000211102C081E329C001968330910510F082
:100D500082E090E09093550180935401809154017A
:100D6000909155018230910529F0019709F04DC00D
:100D700082E0A2CF9091520181E0892780935201B5
:100D800044C0009709F070CF2091520121116CCF1F
:100D900081E312CF80FD8FCF8EE20E94651335C0B4
:100DA00080FD98CF8EE208CF12968C91882311F0A7
:100DB00080EF0FC080EF12C012968C91882311F043
:100DC00080EF15C080EF1AC012968C91882329F00D
:100DD00081EF0E94FC1E82EF0DC081EF0E94641F14
:100DE00082EF0FC012968C91882339F081EF0E9418
:100DF000FC1E83EF0E94FC1E06C081EF0E94641F50
:100E000083EF0E94641F0E94E91F80E090E0089534
:100E100008958091580190915901892B19F0259AD4
:100E20002D9A0DC0E0910E01F0910F01808185FD9A
:100E3000F6CF0E94491281FDF2CF25982D9880911E
:100E4000C60181FF03C0269A2E9A02C026982E98CA
:100E50008091C60182FF03C0279A2F9A0895279890
:100E60002F98089581E0089581E008950C94340747
:100E70000895282F882339F090E02A3010F44D96F9
:100E800008950697089587E290E00895AF92BF9283
:100E9000DF92EF92FF920F931F93CF93DF938C011A
:100EA000FC01C081D181CE010E94DB1BBE010E94EA
:100EB000B60AEC01B8010E943607882309F4C9C1BB
:100EC000F8018281882309F4BEC0809166018111F6
:100ED0001FC0C431F0E7DF0709F0B5C10E94380731
:100EE00081E0809366010E94A91D90936501809323
:100EF000640110925D0110925F0110925E011092E8
:100F00006101109260011092630110926201A1C10F
:100F100080916401909165010E94B51D883C910506
:100F200070F480915D01E82FF0E0EE0FFF1FE25AB0
:100F3000FE4FD183C0838F5F80935D018AC1C13032
:100F400020E8D20708F451C0F8018281882309F40F
:100F50007EC05E01E894B7F880915C01813079F041
:100F600050F08230C1F482EE0E94651387E50E9442
:100F7000651387E50EC082EE0E9465130CC080EEFB
:100F80000E94651381EE0E94651388E10E9465133B
:100F900088E10E942D148CE0E82EF12CC5010E2C66
:100FA00002C0969587950A94E2F78F700E943907E0
:100FB000D82E0E9465138D2D0E942D14F4E0EF1A97
:100FC000F1082CEFE2162FEFF20641F780915C0159
:100FD000813029F010F0823041F482EE04C080EEBE
:100FE0000E942D1481EE0E942D14C43180E7D80791
:100FF00068F4C23090E7D90708F046C0C115E0E7B1
:10100000DE0771F0C130D047A1F10CC1C33320E736
:10101000D20709F4D8C0C433D04709F4EBC002C1E9
:10102000F8018281882309F402C10E94E216FFEFD1
:1010300024E38CE0F15020408040E1F700C0000044
:101040000E94041E06C1C13080E8D80770F2C43186
:1010500020E7D20708F0B3C0C23080E7D807A0F479
:10106000C11590E7D90709F4E2C0C130D04709F0B3
:10107000D9C0F8018281882309F4D9C08091E301A5
:1010800081608093E301E5C0F8018281882309F43F
:10109000CEC00E945E1E811102C00E94441E0E94AA
:1010A000711E90E09093F7018093F601C230F0E753
:1010B000DF0721F48091F60181607AC0C33020E718
:1010C000D20721F48091F601826072C0C43080E7BB
:1010D000D80721F48091F60184606AC0C53090E79A
:1010E000D90719F48091F60127C0C630E0E7DE0782
:1010F00021F48091F60180615BC0C730F0E7DF0723
:1011000021F48091F601806253C0C83020E7D207F5
:1011100021F48091F60180644BC0C93080E7D80784
:1011200021F48091F601806843C0CA3090E7D90766
:1011300029F48091F601846088603AC0CB30E0E702
:10114000DE0721F48091F6018E7F32C0CC30F0E7CB
:10115000DF0721F48091F6018D7F2AC0CD3020E792
:10116000D20721F48091F6018B7F22C0CE3080E738
:10117000D80719F48091F6011AC08091F601CF309A
:1011800090E7D90711F48F7E13C0C031E0E7DE0786
:1011900011F48F7D0DC0C131F0E7DF0711F48F7BB3
:1011A00007C0C231D04711F48F7702C08B7F877F91
:1011B0008093F6018091F6010E94751E4AC0C333E8
:1011C000F0E7DF07A1F4F8018281882321F0109273
:1011D0005A0182E016C080915A01811106C086E250
:1011E0000E94651386E20E942D1482E018C0C43369
:1011F000D047C1F4F8018281882331F010925B015D
:1012000080E20E947C1425C080915B01811106C0A0
:1012100087E20E94651387E20E942D1480E20E94FB
:10122000831417C081E080935A0180935B01C80149
:10123000DF91CF911F910F91FF90EF90DF90BF90C2
:10124000AF900C943207C130F0E8DF0708F081CE90
:10125000CCCE80E0DF91CF911F910F91FF90EF9066
:10126000DF90BF90AF90089526E0729FF0011124A7
:1012700044E5849FE00DF11D1124E60FF11DEE0FF2
:10128000FF1FE65BFE4F859194910E94C80A81156D
:1012900060E49607B0F5811570E3970708F0DEC0AB
:1012A000803E9105D8F4803C910508F06CC0883AE6
:1012B000910578F4853A910508F06BC0813091056D
:1012C00009F452C108F40FC18430910508F04CC1F3
:1012D0000AC18B3B910508F467C005C18F3F91059A
:1012E00009F048F4803F910508F0ADC0883E9105B3
:1012F00008F43AC1F8C0811520E2920708F0A5C0B1
:101300000895811543E5940790F4811562E59607E9
:1013100008F0C8C0811571E5970708F0BEC08115B7
:1013200020E5920708F09DC09F70906A089581158E
:1013300045E59407D8F4811564E5960708F0C8C020
:10134000482F4695469570E2479FA001112483706F
:10135000992721E030E0B90102C0660F771F8A9516
:10136000E2F7CB01842B952B9A680895811576E5D9
:10137000970708F4B2C09C0130562115304108F09F
:10138000B2C09F70AEC0FC01EE0FFF1FEA55F040E7
:1013900062C0853A910509F4A9C0863A910509F021
:1013A000A8C082E890E40895883A910509F4A4C0A1
:1013B000893A910509F4A3C08A3A910509F4A2C0BB
:1013C0008B3A910509F4A1C08C3A910509F4A0C0AB
:1013D0008D3A910509F49FC0803B910509F49EC0A8
:1013E0008E3A910509F49DC08F3A910509F49CC08D
:1013F000813B910509F49BC0823B910509F49AC099
:10140000833B910509F499C0843B910509F498C088
:10141000853B910509F497C0863B910509F496C078
:10142000873B910509F495C0883B910509F494C068
:10143000893B910509F493C08A3B910509F492C058
:1014400080E094E4089590650895FC01FF70EE0F2C
:10145000FF1FEA5DFE4F8591949108959927906C46
:101460000895482F437021E030E002C0220F331F5F
:101470004A95E2F73C68AC0164E0569547956A9559
:10148000E1F74370342B8F708695869560E2869FD6
:10149000C0011124822B932B0895982F8827816FE8
:1014A000906A0895482F4695469570E2479FA0019F
:1014B00011248370992721E030E0B90102C0660F42
:1014C000771F8A95E2F7CB01842B952B9C680895B2
:1014D000982F8827846F906A08958F719927982F85
:1014E00088279062089580E090E0089581E890E474
:1014F000089583E890E4089582EE94E4089589EED7
:1015000094E408958AEE94E4089585EB94E40895B4
:1015100086EB94E4089587EB94E408958CEC94E4CE
:1015200008958DEC94E4089583E895E408958AE89D
:1015300095E4089582E995E4089584E995E4089591
:1015400081E296E4089583E296E4089584E296E4C5
:10155000089585E296E4089586E296E4089587E288
:1015600096E408958AE296E40895089596E0799FB6
:10157000F001112494E5899FE00DF11D1124E60F7F
:10158000F11DEE0FFF1FE65BFE4F859194910895CC
:101590008238910549F1B0F48133910509F458C0BE
:1015A00048F48932910509F44EC08A32910509F454
:1015B00054C008958533910509F440C089339105DD
:1015C00099F00895833E910529F138F4803E910504
:1015D00091F0823E9105A1F00895863E9105F9F0C3
:1015E000873E910531F108952091F60120FD3AC022
:1015F00021FD38C008958091F60180FD35C032C0CC
:101600008091F60182FF32C08091F60184FD30C0E6
:1016100083EE39C08091F60182FD28C0F5CF80911C
:10162000F60183FF27C08091F60184FD21C087EE7B
:101630002AC08091F60183FD1DC0F5CF8091F6018F
:1016400085FD1AC01BC08091F60185FD17C014C02E
:101650008091F60186FD14C015C08091F60186FDCB
:1016600011C00EC080EE0FC089E30DC082EE0BC02A
:1016700080E009C086EE07C089E205C085E303C0AB
:101680008AE201C081E390E0089508950C94450B2F
:10169000809177010895CF93DF9300D01F92CDB74B
:1016A000DEB79C018091FC01843019F593E09983A9
:1016B0003B832A839093E9008FEF9091E80081505B
:1016C00095FD06C095ED9A95F1F700008111F5CFD3
:1016D0008091E80085FF0DC040E050E063E070E0DD
:1016E000CE0101960E94B10D8091E8008E77809323
:1016F000E8000F900F900F90DF91CF910895CF9356
:10170000DF9300D01F92CDB7DEB72091FC012430CB
:1017100021F522E029839B838A8383E08093E9007B
:101720008FEF9091E800815095FD06C095ED9A9558
:10173000F1F700008111F5CF8091E80085FF0DC021
:1017400040E050E063E070E0CE0101960E94B10DF0
:101750008091E8008E778093E8000F900F900F90B3
:10176000DF91CF9108952091FC012430F1F422E023
:101770002093E9002FEF3091E800215035FD06C09D
:1017800035ED3A95F1F700002111F5CF2091E800F1
:1017900025FF0BC040E050E065E070E00E94B10D15
:1017A0008091E8008E778093E8000895CF93DF93CF
:1017B000EC019091FC01943009F046C080910C013D
:1017C0008823D9F080910D018823B9F09093E90026
:1017D0008FEF9091E800815095FD06C095E19A95B4
:1017E000F1F700008111F5CF8091E80085FF2CC052
:1017F00040E050E060E170E017C081E08093E900D4
:101800008FEF9091E800815095FD06C095ED9A9577
:10181000F1F700008111F5CF8091E80085FF14C039
:1018200040E050E068E070E0CE010E94B10D809190
:10183000E8008E778093E80080E1FE01A7E6B1E042
:1018400001900D928A95E1F7DF91CF9108958091F3
:10185000FB01811109C00E94460F0E94A30F8091D5
:10186000E20084608093E20008951092FB010895E5
:1018700008950C94EA220E949A1D0E94F0220E9470
:1018800049120C94460B42E061EC81E00E94C00ECC
:1018900042E061EC82E00E94C00E42E061EC83E035
:1018A0000E94C00E42E161EC84E00C94C00E809175
:1018B000FE01833009F455C030F4813071F082307C
:1018C00009F48EC008958A3009F47AC08B3009F487
:1018D00060C0893009F09CC020C08091FD01813A30
:1018E00009F096C08091E800877F8093E80080919E
:1018F000010290910202892B21F460E187E691E0D8
:1019000003C060E080E090E070E00E94FC0D8091F8
:10191000E8008B778093E80008958091FD01813283
:1019200009F076C08091010290910202009719F0AF
:10193000039709F06DC08091E800877F8093E800ED
:101940008091E80082FD05C08091FC018111F8CFF3
:101950005FC08091F100809377018091E8008B77E0
:1019600053C08091FD01813A09F052C0809101027B
:1019700090910202892B09F04BC08091E800877F8B
:101980008093E8008091E80080FFFCCF80910C01FB
:1019900036C08091FD018132D9F58091010290918C
:1019A0000202892BA9F58091E800877F8093E800E7
:1019B0000E94F50E8091FF0180930C010C94E216B9
:1019C0008091FD01813221F58091E800877F80932D
:1019D000E8000E94F50E809100028093780108953E
:1019E0008091FD01813AA1F48091E800877F809386
:1019F000E8008091E80080FFFCCF8091780180931F
:101A0000F1008091E8008E778093E8000C94F50E49
:101A1000089584B7877F84BF88E10FB6F8948093D8
:101A20006000109260000FBE80E880936100109209
:101A300061000E9498120E94460F0E94A30F80919D
:101A4000E20084608093E20078940E9429120E9450
:101A50009A1282E091E00E9444120E94D822809162
:101A6000FC01853069F40E94621D8091FA0188238F
:101A7000B1F30E948C1D882391F30E949B0DEFCF40
:101A80000E94A012ECCF292F332723303105C9F053
:101A900064F42130310581F02230310509F043C072
:101AA0008DE690E02EE134E042C021323105F1F0C4
:101AB0002232310541F137C082E190E02BE834E079
:101AC00036C099278130910541F08230910541F06F
:101AD000892B49F5EAE1F4E005C0E2E0F4E002C058
:101AE000EAEEF3E0849190E09F0121C06430D8F4E5
:101AF000E62FF0E0EE0FFF1FEE5DFE4F20813181FB
:101B000089E090E014C0643070F470E0FB01EE0FE7
:101B1000FF1FE65EFE4F20813181FB01EA5EFE4F32
:101B2000808190E004C080E090E020E030E0FA01A5
:101B300031832083089580E189BD82E189BD09B4A4
:101B400000FEFDCF8091D8008F7D8093D8008091DA
:101B5000E00082608093E0008091E00081FDFCCF96
:101B60000895CF92DF92EF92FF920F931F93CF933E
:101B7000DF93EC018B016A010E94140F811133C0C5
:101B8000C114D10439F0F60180819181081B190B31
:101B9000C80FD91FE12CF12C0115110519F1809105
:101BA000E80085FD16C08091E8008E778093E800FC
:101BB000C114D10449F0F60180819181E80EF91E2B
:101BC000F182E08285E00FC00E94140F882321F388
:101BD0000AC089918093F10001501109FFEFEF1ABB
:101BE000FF0ADACF80E0DF91CF911F910F91FF9034
:101BF000EF90DF90CF90089520910302309104027E
:101C00002617370748F06115710539F42091E8006F
:101C10002E772093E80001C0B90140E061157105FD
:101C2000A9F12091FC01222309F443C0253009F4D5
:101C300042C02091E80023FD40C02091E80022FD31
:101C400032C02091E80020FFE9CF4091F3002091BD
:101C5000F20030E0342BFC01CF016115710559F021
:101C60002830310540F481918093F1006150710971
:101C70002F5F3F4FF1CF41E02830310509F040E0C0
:101C80002091E8002E772093E800C8CF4111C9CFFA
:101C90000AC08091FC01882361F0853061F0809159
:101CA000E80083FD0AC08091E80082FFF2CF80E067
:101CB000089582E0089583E0089581E008952091D9
:101CC0000302309104022617370748F061157105A9
:101CD00039F42091E8002E772093E80001C0B90183
:101CE000FC0120E06115710591F18091FC018823D0
:101CF00009F440C0853009F43FC08091E80083FDBD
:101D00003DC08091E80082FD2FC08091E80080FFF7
:101D1000E9CF2091F3008091F20090E0922B6115C1
:101D2000710559F08830910540F424912093F10019
:101D30003196615071090196F2CF21E0089709F0C0
:101D400020E08091E8008E778093E800CBCF2111CE
:101D5000CCCF0AC08091FC01882361F0853061F00E
:101D60008091E80083FD0AC08091E80082FFF2CFF5
:101D700080E0089582E0089583E0089581E0089569
:101D8000982F973058F59093E900981739F0709193
:101D9000EC002091ED005091F00003C0242F762F2D
:101DA00050E021FF19C03091EB003E7F3093EB00F3
:101DB0003091ED003D7F3093ED003091EB003160CC
:101DC0003093EB007093EC002093ED005093F00003
:101DD0002091EE0027FF07C09F5FD3CF8F708093C5
:101DE000E90081E0089580E008958091FD0187FF7A
:101DF00011C08091E80082FD05C08091FC01811135
:101E0000F8CF11C08091E8008B770BC08091FC0166
:101E1000882349F08091E80080FFF8CF8091E800A6
:101E20008E778093E80008952091E4003091E500DA
:101E300095E64091EC00842F817040FF22C0809194
:101E4000E80080FD1CC08091FC01882391F0853062
:101E500091F08091EB0085FD10C04091E40050911D
:101E6000E5004217530729F39A01915011F784E0D6
:101E7000089582E0089583E0089581E0089580E068
:101E800008954091E80042FFDECF08950E94B40F0C
:101E90000E94BC0FE0EEF0E0808181608083E8ED7D
:101EA000F0E080818F77808319BCA7EDB0E08C9142
:101EB0008E7F8C9380818F7E80831092FB010895AA
:101EC0000F931F93CF93DF930E94B40F0E94BC0F18
:101ED000C8EDD0E088818F77888388818068888387
:101EE00088818F7D888319BC1092FC011092F801C3
:101EF0001092FA011092F90100EE10E0F8018081D1
:101F00008B7F808388818160888342E060E080E00D
:101F10000E94C00EE1EEF0E080818E7F8083E2EED1
:101F2000F0E0808181608083808188608083F80117
:101F300080818E7F8083888180618883DF91CF91CB
:101F40001F910F910895E8EDF0E080818F7E8083EE
:101F5000E7EDF0E080818160808384E082BF81E0F2
:101F60008093FB010C94600FE8EDF0E080818E7FA0
:101F700080831092E20008951092DA001092E1003E
:101F800008951F920F920FB60F9211242F933F9333
:101F90004F935F936F937F938F939F93AF93BF9371
:101FA000EF93FF938091E10082FF0BC08091E200EC
:101FB00082FF07C08091E1008B7F8093E1000E9447
:101FC00028128091DA0080FF1FC08091D80080FF26
:101FD0001BC08091DA008E7F8093DA008091D90057
:101FE00080FF0DC080E189BD82E189BD09B400FE9A
:101FF000FDCF81E08093FC010E94270C05C019BC35
:102000001092FC010E94350C8091E10080FF19C004
:102010008091E20080FF15C08091E2008E7F809366
:10202000E2008091E20080618093E2008091D8001C
:1020300080628093D80019BC85E08093FC010E94E7
:10204000390C8091E10084FF30C08091E20084FF70
:102050002CC080E189BD82E189BD09B400FEFDCFBD
:102060008091D8008F7D8093D8008091E1008F7E91
:102070008093E1008091E2008F7E8093E200809166
:10208000E20081608093E2008091F801882311F0E2
:1020900084E007C08091E30087FD02C081E001C0B9
:1020A00083E08093FC010E943B0C8091E10083FF60
:1020B00029C08091E20083FF25C08091E100877FE5
:1020C0008093E10082E08093FC011092F8018091FE
:1020D000E1008E7F8093E1008091E2008E7F80930B
:1020E000E2008091E20080618093E20042E060E0E3
:1020F00080E00E94C00E8091F00088608093F00024
:102100000E94380CFF91EF91BF91AF919F918F91F9
:102110007F916F915F914F913F912F910F900FBEE3
:102120000F901F9018951F920F920FB60F921124C7
:102130002F933F934F935F936F937F938F939F93CF
:10214000AF93BF93CF93DF93EF93FF93C091E900D9
:10215000CF708091EC00D82FD17080FDD0E8109224
:10216000E9008091F000877F8093F00078940E94CE
:10217000D7101092E9008091F00088608093F00001
:10218000CD2BCF70C093E900FF91EF91DF91CF91FC
:10219000BF91AF919F918F917F916F915F914F917F
:1021A0003F912F910F900FBE0F901F9018951F9386
:1021B000CF93DF93CDB7DEB7AA970FB6F894DEBF03
:1021C0000FBECDBFEDEFF1E088E08E0F9091F100F2
:1021D00091938E13FBCF0E94570C8091E80083FFF0
:1021E0001FC18091FD019091FE01492F50E04A30BE
:1021F000510508F015C1FA01EC59FF4F0C947224F7
:10220000803881F0823809F00BC1809101028F7013
:102210008093E9008091EB0085FB882780F910927C
:10222000E90006C08091F9019091FA019111826054
:102230009091E800977F9093E8008093F1001092CE
:10224000F100C8C0282F2D7F09F0EAC0882319F0BB
:10225000823061F0E5C08091FF01813009F0E0C07B
:10226000933009F080E08093FA012BC08091FF0148
:10227000811127C0809101028F7009F4D1C0809331
:10228000E9002091EB0020FF1CC0933021F48091E5
:10229000EB00806214C09091EB0090619093EB0092
:1022A00021E030E0A90102C0440F551F8A95E2F7F2
:1022B0004093EA001092EA008091EB0088608093DE
:1022C000EB001092E9008091E800877F86C08111C1
:1022D000A7C01091FF011F778091E3008078812BC8
:1022E0008093E3008091E800877F8093E8000E945C
:1022F000F50E8091E80080FFFCCF8091E3008068BC
:102300008093E300111102C082E001C083E080935A
:10231000FC0186C08058823008F082C08091FF01A5
:10232000909100028C3D53E0950779F583E08A8314
:102330008AE289834FB7F894DE01139620E03EE0ED
:1023400051E2E32FF0E050935700E49120FF03C0E7
:10235000E295EF703F5FEF708E2F90E0EA3010F063
:10236000C79601C0C0968D939D932F5F243149F786
:102370004FBF8091E800877F8093E8006AE270E0B9
:10238000CE0101960E94FC0D14C0AE014F5F5F4F5D
:10239000609101020E94430DBC01009709F440C006
:1023A0009091E800977F9093E80089819A810E943C
:1023B0005F0E8091E8008B778093E80031C0803811
:1023C00079F58091E800877F8093E8008091F8019B
:1023D0008093F1008091E8008E778093E8000E945E
:1023E000F50E1EC081111CC09091FF019230C0F407
:1023F0008091E800877F8093E8009093F8010E9425
:10240000F50E8091F801811106C08091E30087FDEF
:1024100002C081E001C084E08093FC010E94430C73
:102420008091E80083FF0AC08091E800877F809355
:10243000E8008091EB0080628093EB00AA960FB6D3
:10244000F894DEBF0FBECDBFDF91CF911F910895ED
:102450000895CF938091FC018823A1F0C091E900F9
:10246000CF709091EC00892F817090FD80E8C82B8F
:102470001092E9008091E80083FD0E94D710CF7090
:10248000C093E900CF91089590937E0180937D01E0
:102490000895E0917D01F0917E01309721F0019047
:1024A000F081E02D099480E00895E0917D01F091A4
:1024B0007E01309721F00280F381E02D0994089588
:1024C000E0917D01F0917E01309721F00480F5814B
:1024D000E02D0994089520917B0130917C018217B1
:1024E000930771F090937C0180937B01E0917D01D3
:1024F000F0917E01309721F00680F781E02D09945C
:1025000008952091790130917A018217930771F033
:1025100090937A0180937901E0917D01F0917E01A1
:10252000309721F00084F185E02D099408950895F5
:102530000C9497120E94A01D0E94AD030C94261EBD
:102540009F92AF92BF92CF92DF92EF92FF920F9342
:102550001F93CF93DF9300D000D000D0CDB7DEB76C
:102560000E94D4030DE010E0AA24A394B12C902E75
:10257000802F0E94C204980120583E4F6901F90142
:10258000F080F826A1F40150110988F78FEF8983B4
:102590008A831B820E94A91D8160782F9D838C8372
:1025A00049815A816B818D810E9437132FC0909190
:1025B000E30191FF04C08E830E94C8048E8125E050
:1025C00030E0A501022E01C0440F0A94EAF7E42E80
:1025D0004F21C1F029839A828E2191E009F490E085
:1025E0009B830E94A91D8160782F9D838C834981E4
:1025F0005A816B818D810E943713F6018081E82614
:10260000E08204C021503109E0F6BDCF0E94F41FE2
:1026100010917F010E9449121817B9F00E944912C7
:1026200080937F0126960FB6F894DEBF0FBECDBF14
:10263000DF91CF911F910F91FF90EF90DF90CF909E
:10264000BF90AF909F900C94460B26960FB6F894CF
:10265000DEBF0FBECDBFDF91CF911F910F91FF90D5
:10266000EF90DF90CF90BF90AF909F900895CF9361
:10267000DF93CDB7DEB72B970FB6F894DEBF0FBE52
:10268000CDBF4F83588769877A878B87DE01119684
:1026900086E0FD0111928A95E9F785E0FE01379603
:1026A00001900D928A95E1F749815A816B817C8175
:1026B0008D819E810E9480192B960FB6F894DEBF03
:1026C0000FBECDBFDF91CF910895CF93882309F43A
:1026D000C2C0C82F823859F40E94491281FDBBC084
:1026E00089E30E945A1C0E94271D89E30CC083388D
:1026F00079F40E94491280FDAEC083E50E945A1C05
:102700000E94271D83E50E949C1CCF910C94271DDD
:10271000843859F40E94491282FD9DC087E40E94CA
:102720005A1C0E94271D87E4EECF8CEF8C0F813A54
:1027300048F48C2F0E943E2281118DC08C2F0E9464
:102740005A1CE3CF80E28C0F883048F4C77081E0D8
:1027500001C0880FCA95EAF70E94E01CD6CF8BE52E
:102760008C0F833078F4C53A29F0C63A31F083E80B
:1027700090E005C081E890E002C082E890E0CF914F
:102780000C946B1288E58C0F833108F064C0C83A52
:1027900039F1C93A41F1CA3A49F1CB3A51F1CC3A4F
:1027A00059F1CD3A61F1C03B69F1CE3A71F1CF3ABE
:1027B00079F1C13B81F1C23B89F1C33B91F1C43B4B
:1027C00099F1C53BA1F1C63BA9F1C73BB1F1C83BAB
:1027D000B9F1C93BC1F1CA3BC9F180E090E038C012
:1027E00082EE90E035C089EE90E032C08AEE90E053
:1027F0002FC085EB90E02CC086EB90E029C087EBE2
:1028000090E026C08CEC90E023C08DEC90E020C0DE
:1028100083E891E01DC08AE891E01AC082E991E066
:1028200017C084E991E014C081E292E011C083E214
:1028300092E00EC084E292E00BC085E292E008C014
:1028400086E292E005C087E292E002C08AE292E06E
:10285000CF910C948112CF910895882309F44BC035
:10286000823859F40E94491281FF45C089E30E94D1
:102870005A1C0E94271D89E30CC0833871F40E9402
:10288000491280FF38C083E50E945A1C0E94271D10
:1028900083E50E949C1C0C94271D843859F40E94E7
:1028A000491282FF28C087E40E945A1C0E94271DFB
:1028B00087E4EFCF9CEF980F913A58F390E2980F8E
:1028C000983050F4877091E001C0990F8A95EAF72B
:1028D000892F0E94E61CDFCF9BE5980F933020F4F0
:1028E00080E090E00C946B12885A833120F480E0F1
:1028F00090E00C9481120895882321F00E94E01C3E
:102900000C94271D0895882321F00E94E61C0C9446
:10291000271D08957F928F929F92AF92BF92CF9280
:10292000DF92EF92FF920F931F93CF93DF931F924B
:10293000CDB7DEB77C01C62E772EFC01058102954E
:102940000F70128111110E94FD1C0E94531C8823DC
:1029500079F0112369F080E28C0D883048F082E034
:102960000E943C1C0E94531C91E0D82ED92601C025
:10297000D12CE72DE295EF70F0E0E259FF4F0C9477
:102980007224872D807F072D0F70882311F0029508
:10299000007F112389F0002309F490C180E28C0D9F
:1029A000883020F4802F0E94E01C03C0802F0E94FA
:1029B000F01C0E94271D82C18C2D0E942D14002323
:1029C00009F495C180E28C0D883020F4802F0E949C
:1029D000E61C03C0802F0E94F61C0E94271D87C1A1
:1029E000972D907F872D8F70903211F08295807F88
:1029F000CC2021F0F1E0CF16B1F01EC0112349F038
:102A0000002309F414C1013009F011C10E94101D06
:102A10006EC1002319F0013009F469C189830E9455
:102A2000131D89810AC1112321F0023008F05FC112
:102A3000FEC001115CC101C1112321F0002309F482
:102A4000F6C03CC1002309F4F8C03EC1872D86952D
:102A50008695837090E0009719F0019761F047C167
:102A6000112321F08C2D972D937002C080E090E00F
:102A70000E946B123CC1112321F08C2D972D937075
:102A800002C080E090E00E94811231C18C2D1123A0
:102A900019F00E94FC1E02C00E94641F0E94E91FE0
:102AA00026C1872D837009F052C0111120C18C2DD1
:102AB000829586958770880F880F9C2D9F70892E30
:102AC000912CA12CB12C082E04C0880C991CAA1C96
:102AD000BB1C0A94D2F7C4FE14C00FE010E020E043
:102AE00030E0B901A80104C0440F551F661F771FCD
:102AF0008A95D2F7CB01BA01609570958095909533
:102B000003C060E070E0CB01272D26952695237049
:102B100030E02230310569F02330310589F0682931
:102B200079298A299B292130310571F00E94C81A20
:102B3000DEC0682979298A299B290E94E41AD7C016
:102B40000E94C81AC501B4010E94AC1AD0C011235A
:102B500019F0872D817001C08695882309F4C7C0BC
:102B60008C2D829586958770880F880F9C2D9F707D
:102B7000892E912CA12CB12C082E04C0880C991CF4
:102B8000AA1CBB1C0A94D2F7C4FE14C00FE010E0CC
:102B900020E030E0B901A80104C0440F551F661FB2
:102BA000771F8A95D2F7CB01BA0160957095809511
:102BB000909503C060E070E0CB01272D2695269507
:102BC0002370422F50E04230510569F043305105E7
:102BD00089F0682979298A299B294130510571F0AA
:102BE0000E94A21B84C0682979298A299B290E94F6
:102BF000BE1B7DC00E94A21BC501B4010E94861BA2
:102C000076C08C2D90E0FC01E05EF109E531F10524
:102C100008F050C0E258FF4F0C9472240C2D0F7036
:102C2000872D8F71112331F00E941F1B802F0E946E
:102C30007C145DC00E94401B802F0E94831457C0EB
:102C4000112339F0011153C0872D8F710E94651B2C
:102C50004EC0023008F04BC0F7CF112339F0872D5A
:102C60008F710E941F1B43C01123C9F3872D8F71E1
:102C70000E94401B3CC0112329F0872D8F710E94B8
:102C80000A1B35C00E94001B32C0112351F0172DC2
:102C90001F71812F0E941F1B63E0812F0E94331C34
:102CA00026C081E00E943C1C023008F182E00E94B4
:102CB0003C1C1DC0112331F0002389F28C2D0E9491
:102CC000651315C0002391F28C2D0E942D140FC0A6
:102CD000472D4F706C2DC7010E949E050E94241A3B
:102CE00006C0472D4F706C2DC7010E94B50ADD202C
:102CF000F9F00E942F1C80FD1BC0F70112820E9478
:102D0000291C0E941F1BC7010E94A7160E94291C94
:102D10000F90DF91CF911F910F91FF90EF90DF9077
:102D2000CF90BF90AF909F908F907F900C94401B5E
:102D30000F90DF91CF911F910F91FF90EF90DF9057
:102D4000CF90BF90AF909F908F907F9008950F93FA
:102D50001F93CF93DF93EC01888199812B813C8174
:102D6000232BB9F09F3F11F48F3F99F0CE010E94C1
:102D70004607882371F0688179818A810E94251C29
:102D80008C010E94DA1B0E94A11AB801CE010E9498
:102D90008A14DF91CF911F910F9108950E94FD1C1D
:102DA0000E940D1D0E94D21C0E94271D0E949A2085
:102DB0000E94E91F80E090E00E946B1280E090E0AA
:102DC0000C9481120E94ED1C0C94CE160E941A1CC9
:102DD000292F22952F7030E02C3031054CF42A3009
:102DE00031056CF42250310922303105A8F407C0B6
:102DF0002C30310569F02F30310551F00DC0803F86
:102E000069F018F4803E40F409C0843F29F406C0FC
:102E100093FB882780F9089580E0089581E0089564
:102E2000CF93DF9300D000D01F92CDB7DEB70F90C5
:102E30000F900F900F900F90DF91CF910895CF9347
:102E4000DF9300D000D000D0CDB7DEB726960FB606
:102E5000F894DEBF0FBECDBFDF91CF9108951F93D1
:102E6000CF93DF93C0918E0116E080918F01C81738
:102E700099F0D0E01C9FF0011D9FF00D1124E05748
:102E8000FE4F4081518162817381848195810E94CE
:102E90001F172196C770E9CFDF91CF911F91089539
:102EA0004091C0015091C1016091C2017091C30174
:102EB0008091C4019091C5010C941F178091C501A8
:102EC00082958F7009F054C08091C201882309F463
:102ED0004FC080918E01A0918F016091C0017091CF
:102EE000C1014091C3015091C401B6E08A1709F4B1
:102EF0003FC090E041155105C1F17F3F11F46F3F94
:102F0000A1F1B89FF001B99FF00D1124E057FE4FD9
:102F1000218172132AC02081621327C022812111CE
:102F200024C0238134812417350710F4215031093E
:102F3000241B350B283C3105C0F42091C5012F70AE
:102F400020612093C50126E0289FF001299FF00D04
:102F50001124EB56FE4F80818F708061808380EC5E
:102F600091E00E94A7160C942F1701968770BECF90
:102F70000895CF92DF92EF92FF920F931F93CF931A
:102F8000DF93CDB7DEB762970FB6F894DEBF0FBE02
:102F9000CDBF8C0185E0F801DE011D9601900D92F8
:102FA0008A95E1F7D8014C9111965C911197129690
:102FB0006C9112971396CD90DC9014973091C001CC
:102FC0007091C1018091C3019091C401009709F4EF
:102FD0006BC17F3F19F43F3F09F466C1E090C20125
:102FE000EE2009F4C0C02091C501C816D90628F00A
:102FF000F601E81BF90BCF0104C0809590958C0D6C
:103000009D1DFF24F394883C910578F0F12C207FDE
:1030100009F0C6C07C2DD98AC88A89890E941017F8
:1030200080EC91E00E94A716B1C0822F807F09F04A
:1030300046C0751314C0341312C0611110C02F7034
:1030400020612093C5010E94501780EC91E00E94FE
:10305000A7168091C501D80115968C932EC0CD2856
:1030600019F15F3F11F44F3FF9F0F62E61111CC0CA
:1030700080918E0120918F0136E0821709F45AC0A9
:1030800090E0389FF001399FF00D1124E057FE4F7A
:103090007181571306C07081471303C0728171118B
:1030A00003C001968770E9CFF62E662309F418C194
:1030B0008091C50181608093C501F12C11C1751308
:1030C00008C0341306C0611104C08091C501D80145
:1030D000C3C04D875E878D859E856A8B0E94E616EC
:1030E0006A898823E1F16623D1F12091C501822FFD
:1030F00082958F7090E0029774F08091C00190915A
:10310000C10198878F831986DB86CA862C87CE01FA
:1031100007960E94A71686E0F801A0ECB1E00190A6
:103120000D928A95E1F70E945E170E945017FF24C6
:10313000F394D6C04D875E878D859E850E941A1CAC
:10314000292F22952F7030E0223031050CF0BCC0C1
:103150009F7009F0B6C0805E883008F4C1C0C80115
:103160000E94A716E4CFC816D90608F453C0F6018A
:10317000E81BF90BCF01883C910508F450C0F12CF5
:103180007C2DD98AC88A89890E941017E0ECF1E069
:1031900086E0DF011D928A95E9F70E945017A0C0D2
:1031A000751314C0341312C0611110C08091C50191
:1031B000F8018583C8010E94A71686E0E0ECF1E0E3
:1031C000DF011D928A95E9F7FE2C8AC04D875E8744
:1031D0008D859E856A8B0E94E6166A89882309F48C
:1031E000BECF662309F4BBCF2091C501822F829503
:1031F0008F7090E002970CF48ECF8091C001909177
:10320000C1019A8389831B82DD82CC822E83CE0109
:1032100001967FCF809590958C0D9D1DACCFF62E9D
:10322000662309F49CCF75132EC034132CC0209153
:10323000C50120FD1FC0822F82958F70D9F0D80163
:1032400015962C9315978F3049F08F5F982F929594
:10325000907F822F8F70892B15968C93C8010E94C6
:10326000A71686E0F801A0ECB1E001900D928A95D6
:10327000E1F793CF86E0F801A0ECB1E001900D9268
:103280008A95E1F72DC04D875E878D859E850E94CA
:10329000E616811140CF8091C50181608093C50100
:1032A000C8010E94A7161CC0662309F458CF4D8799
:1032B0005E878D859E850E94E616882309F44FCF90
:1032C0002ACF811148CF0CC0243031050CF047CFF4
:1032D0009F7009F440CFF8019581907F09F03BCFB2
:1032E0008F2D62960FB6F894DEBF0FBECDBFDF9173
:1032F000CF911F910F91FF90EF90DF90CF900895A5
:103300001F93CF93DF93CDB7DEB72C970FB6F8940A
:10331000DEBF0FBECDBF4F83588769877A878B8703
:103320009C87CE0107960E94B917882369F08F8188
:1033300098852A853B85232BF1F19F3F09F063C0D7
:103340008F3F09F060C037C086E0FE013796DE018E
:10335000119601900D928A95E1F76F817885EA8543
:10336000FB85309741F17F3F11F46F3F21F12091B0
:103370008F0130E0C90101968770992740918E0135
:1033800050E08417950709F447C069837A83FD8369
:10339000EC8396E0929FD001939FB00D1124A0572B
:1033A000BE4FFE01319601900D929A95E1F7809300
:1033B0008F010E942F1716E080918E0190918F014E
:1033C0008917C1F1189FC001112480579E4F0E9498
:1033D000B917882379F1E0918E011E9FF001112425
:1033E000E057FE4F408151816281738184819581D4
:1033F0000E941F1780918E0190E001968770992797
:1034000080938E01D9CF4F81588569857A858B85C8
:103410009C850E941F17CFCF0E94E21610928F0149
:1034200010928E01E0ECF1E086E0DF011D928A95BA
:10343000E9F7C1CF2C960FB6F894DEBF0FBECDBF13
:10344000DF91CF911F910895EF92FF920F931F93F9
:10345000CF93DF938C01009709F46CC0F12CEE241C
:10346000E394E8012196F8018491843740F4843094
:1034700008F051C0813081F0823019F15BC085378E
:1034800009F444C0A8F19CE7980F903708F052C0A7
:103490008F770E942D1441C00E5F1F4FFE01C49113
:1034A00080E28C0F883048F4C7708E2D01C0880FE1
:1034B000CA95EAF70E94001D14C08C2F0E94651364
:1034C0002DC00E5F1F4FFE01C49180E28C0F88302B
:1034D00058F4C7708E2D01C0880FCA95EAF70E9474
:1034E000061D0E94271D1AC08C2F0E942D1416C085
:1034F0000E5F1F4FFE01C491CC2381F08FE99FE046
:103500000197F1F700C00000C150F6CF0E5F1F4FCA
:10351000FE01F49003C00E9465138E018F2D882355
:1035200009F49FCFEFE9FFE03197F1F700C0000009
:103530008150F5CFDF91CF911F910F91FF90EF90C8
:10354000089508956093CA017093CB018093CC01D4
:103550009093CD010C94CE160F931F930091CA0146
:103560001091CB012091CC013091CD01DC01CB0138
:10357000802B912BA22BB32B8093CA019093CB016C
:10358000A093CC01B093CD011F910F910C94CE1656
:103590000F931F930091CA011091CB012091CC0190
:1035A0003091CD01DC01CB0180239123A223B323F1
:1035B0008093CA019093CB01A093CC01B093CD012D
:1035C0001F910F910C94CE160F931F930091CA0177
:1035D0001091CB012091CC013091CD01DC01CB01C8
:1035E00080279127A227B3278093CA019093CB010C
:1035F000A093CC01B093CD011F910F910C94CE16E6
:103600001092C6011092C7011092C8011092C90110
:103610000C94CE1641E050E060E070E004C0440F2E
:10362000551F661F771F8A95D2F74093C6015093A6
:10363000C7016093C8017093C9010C94CE1641E094
:1036400050E060E070E004C0440F551F661F771F14
:103650008A95D2F78091C6019091C701A091C801C7
:10366000B091C901482B592B6A2B7B2B4093C60183
:103670005093C7016093C8017093C9010C94CE1692
:1036800041E050E060E070E004C0440F551F661F49
:10369000771F8A95D2F740955095609570958091E7
:1036A000C6019091C701A091C801B091C9014823FA
:1036B00059236A237B234093C6015093C70160932B
:1036C000C8017093C9010C94CE1641E050E060E04F
:1036D00070E004C0440F551F661F771F8A95D2F70C
:1036E0008091C6019091C701A091C801B091C90114
:1036F000482759276A277B274093C6015093C70163
:103700006093C8017093C9010C94CE160F931F9358
:103710000091C6011091C7012091C8013091C901E3
:10372000DC01CB01802B912BA22BB32B8093C60104
:103730009093C701A093C801B093C9011F910F9145
:103740000C94CE160F931F930091C6011091C701E0
:103750002091C8013091C901DC01CB018023912364
:10376000A223B3238093C6019093C701A093C801FD
:10377000B093C9011F910F910C94CE160F931F9314
:103780000091C6011091C7012091C8013091C90173
:10379000DC01CB0180279127A227B3278093C601A4
:1037A0009093C701A093C801B093C9011F910F91D5
:1037B0000C94CE160895CF92DF92EF92FF920F9362
:1037C0001F93CF93DF938C01C090CA01D090CB019F
:1037D000E090CC01F090CD018091C6019091C7019D
:1037E000A091C801B091C901C82AD92AEA2AFB2AA6
:1037F000CFE1D0E0D701C6010C2E04C0B695A79545
:10380000979587950A94D2F780FF06C0B8018C2F50
:103810000E943409019721F4219760F780E001C0EC
:103820008C2FDF91CF911F910F91FF90EF90DF9040
:10383000CF900895CF93DF93EC010E94DB1BBE0174
:103840000E943409DF91CF910895CB010E941A1C88
:1038500008958091CE0185958595859508958091EF
:10386000CE018770089598E0899F90011124262B3E
:103870002093CE010C941F1B2091CE0180958223B2
:103880008093CE01982F977069F430E0482F552728
:1038900047FD50952417350729F085958595859521
:1038A0000C94401B08959091CE01977081E009F42B
:1038B00080E0089590910C01992321F090910D01E1
:1038C000911109C020910E0130910F01F90132963A
:1038D0009FEF40E01FC0982F9695969596959F3044
:1038E00050F5E0910E01F0910F01E90FF11D877085
:1038F00021E030E0A90102C0440F551F8A95E2F78C
:10390000CA019181892B818308959F3F39F04F5FD0
:103910004E3041F051915813F8CF0DC05111F7CFEF
:10392000942FF5CF9F3F39F0F901E90FF11D97FD75
:10393000FA9582830895089590910C01992321F0BE
:1039400090910D01911109C020910E0130910F014C
:10395000F9013296205F3F4F1FC0982F969596959C
:1039600096959F30F0F4E0910E01F0910F01E90F70
:10397000F11D877021E030E0A90102C0440F551FFE
:103980008A95E2F7CA018095918189238183089500
:103990003196E217F30729F090819813F9CF10823E
:1039A000F7CF089581E090E0E0910E01F0910F01D2
:1039B000E80FF91F1082019680319105A9F708954B
:1039C0009091E201892B8093E20108958095909176
:1039D000E20189238093E20108951092E2010895A3
:1039E0009091E101892B8093E10108958095909158
:1039F000E10189238093E10108951092E101089586
:103A00009091E001892B8093E00108958095909139
:103A1000E00189238093E00108951092E001089568
:103A20008093CF0108951092CF01089580910E01E7
:103A300090910F01FC0131969C01205F3F4F80E087
:103A4000919191118F5FE217F307D1F70895E091FB
:103A50000E01F0910F018091E2018083E0910E014F
:103A6000F0910F0190818091E101892B8083E09199
:103A70000E01F0910F0190818091E001892B8083EC
:103A80008091CF01882361F0E0910E01F0910F0148
:103A90009081892B80830E94161D81111092CF0185
:103AA00080910E0190910F010C94551220E0009727
:103AB00039F0AC0141505109842395232F5FF7CF92
:103AC000822F08958091FC01843021F11092E4014D
:103AD00020E488E190E00FB6F894A8958093600008
:103AE0000FBE2093600080E00E94460B83B7817F69
:103AF000846083BF83B7816083BF7894889583B7E0
:103B00008E7F83BF88E10FB6F89480936000109297
:103B100060000FBE089508950E94C1030E94D4035F
:103B20000E948B1D0E94C90491E0811101C090E0A8
:103B3000892F08950E94E2160E9449120C94460BA8
:103B400082E084BD93E095BD9AEF97BD80936E00AF
:103B500008952FB7F8948091E5019091E601A09126
:103B6000E701B091E8012FBF0895CF92DF92EF9265
:103B7000FF920F931F932FB7F8944091E501509156
:103B8000E6016091E7017091E8012FBF6A017B01B6
:103B9000EE24FF248C0120E030E0C016D106E206BE
:103BA000F30610F4415051099A01281B390BC90141
:103BB0001F910F91FF90EF90DF90CF9008951F928B
:103BC0000F920FB60F9211248F939F93AF93BF93D1
:103BD0008091E5019091E601A091E701B091E801A3
:103BE0000196A11DB11D8093E5019093E601A0937C
:103BF000E701B093E801BF91AF919F918F910F9032
:103C00000FBE0F901F9018950E94460FF8942FEF4B
:103C100087EA91E6215080409040E1F700C0000023
:103C200087E090EBDC018093050290930602A0935D
:103C30000702B09308029CE088E10FB6F894A895BB
:103C4000809360000FBE90936000FFCF0E945E1EC5
:103C5000811102C00E94441E0E94691E8093E301EC
:103C60000E94711E90E09093F7018093F60187FB0C
:103C7000882780F980930D010E946D1E682F70E0E7
:103C800080E090E00C94A21A6DEE7EEF80E090E070
:103C90000E94AC2460E082E090E00E949A2460E000
:103CA00083E090E00E949A2460E084E090E00E942B
:103CB0009A2460E085E090E00C949A2480E090E003
:103CC0000E94942421E08D3E9E4F09F020E0822F37
:103CD000089582E090E00C948C2483E090E00C94B2
:103CE0008C2484E090E00C948C24682F84E090E095
:103CF0000C949A248091EB0180FF0BC0609113011A
:103D000085E0689FB0011124759567957595679555
:103D10002BC081FF09C06091130185E0689FB0014D
:103D200011247595679520C082FF07C0609113012B
:103D300085E0689FB001112417C09091EC01992390
:103D4000D1F060911201961788F72091130185E058
:103D5000289F90011124929FA001939F500D112440
:103D600070E0CA010E945E246038710540F461155C
:103D7000710539F002C065E070E0862F08958FE785
:103D8000089581E008958091EB0180FF08C0609163
:103D9000110170E0759567957595679521C081FF54
:103DA00006C06091110170E07595679519C082FF9A
:103DB00004C06091110170E010C09091EC01992352
:103DC000C1F0609110019617A0F780911101899FB1
:103DD000C001112470E00E945E246038710528F44F
:103DE0006115710521F0862F08958FE7089581E010
:103DF000089561E070E0F4CF803F21F40E947A1EC4
:103E0000819504C0813F29F40E947A1E8093EF01BE
:103E10000895823F21F40E947A1E819504C0833F59
:103E200029F40E947A1E8093EE010895893F19F4C7
:103E30000E94C31E05C08A3F31F40E94C31E8195B3
:103E40008093F00108958B3F21F40E94C31E819559
:103E500004C08C3F29F40E94C31E8093F101089591
:103E6000843F21F48091ED01816017C0853F21F4EA
:103E70008091ED01826011C0863F21F48091ED01B7
:103E800084600BC0873F21F48091ED01886005C0FC
:103E9000883F31F48091ED0180618093ED010895B8
:103EA0008D3F21F48091EB0181600BC08E3F21F4A6
:103EB0008091EB01826005C08F3F29F48091EB0176
:103EC00084608093EB010895803F39F48091EF0185
:103ED00087FF6CC01092EF0169C0813F29F4809187
:103EE000EF011816BCF362C09091EE01823F29F4F5
:103EF00097FF5CC01092EE0159C0833F19F4191668
:103F0000CCF354C0893F41F48091F00118160CF0B5
:103F10004DC01092F0014AC08A3F29F48091F0010F
:103F200087FF44C0F6CF8B3F39F48091F10187FFC2
:103F30003DC01092F1013AC08C3F29F48091F1010B
:103F40001816BCF333C0843F21F48091ED018E7FBD
:103F500017C0853F21F48091ED018D7F11C0863F10
:103F600021F48091ED018B7F0BC0873F21F480917C
:103F7000ED01877F05C0883F31F48091ED018F7E90
:103F80008093ED0113C08D3F21F48091EB018E7F72
:103F90000BC08E3F21F48091EB018D7F05C08F3FD8
:103FA00029F48091EB018B7F8093EB018091EE01EE
:103FB00081110EC08091EF0181110AC08091F00142
:103FC000811106C08091F101811102C01092EC01B3
:103FD00008958DEE91E00E9460120E94A91D9093B9
:103FE000EA018093E90108951F93CF93DF938091B5
:103FF000E9019091EA010E94B51DAC019091EC019C
:10400000992321F02091140130E006C02091150180
:104010008AE0289F900111244217530708F486C0B4
:104020008091EE01C091EF01D091F0011091F1016A
:10403000811107C0C11176C0D11174C0111172C0B5
:1040400075C09F3F19F09F5F9093EC01181624F400
:104050000E947A1E8093EE018091EE0187FF05C0D9
:104060000E947A1E81958093EE011C1624F40E9412
:104070007A1E8093EF018091EF0187FF05C00E94B7
:104080007A1E81958093EF016091EE01662339F1EC
:10409000C091EF01CC2319F1772767FD7095872F29
:1040A000972F0E946F2323E333E343E35FE30E94F0
:1040B000D3230E943C236093EE016C2F772767FD8A
:1040C0007095872F972F0E946F2323E333E343E3F9
:1040D0005FE30E94D3230E943C236093EF011D16EF
:1040E00024F40E94C31E8093F0018091F00187FFA9
:1040F00005C00E94C31E81958093F001111624F41F
:104100000E94C31E8093F1018091F10187FF05C0D9
:104110000E94C31E81958093F101DF91CF911F9181
:104120000C94E91F9F3F09F08ECF96CFDF91CF917E
:104130001F910895EDEEF1E085E0DF011D928A9573
:10414000E9F71092EC011092EB010895833081F1B0
:1041500028F4813059F08230D1F00895853009F487
:1041600049C0B8F1863009F456C008958091150110
:10417000262F30E0280F311D2F3F310524F4680F22
:104180006093150108958FEF809315010895809134
:104190001401262F30E0280F311D2F3F310524F464
:1041A000680F6093140108958FEF809314010895B0
:1041B00080911301262F30E0280F311D2F3F31054C
:1041C00024F4680F6093130108958FEF8093130117
:1041D000089580911201262F30E0280F311D2F3FC6
:1041E000310524F4680F6093120108958FEF8093D6
:1041F0001201089580911101262F30E0280F311D02
:104200002F3F310524F4680F6093110108958FEF5B
:1042100080931101089580911001262F30E0280F1E
:10422000311D2F3F310524F4680F6093100108956C
:104230008FEF809310010895833011F128F48130BD
:1042400049F0823091F00895853081F120F1863077
:10425000C1F1089580911501681720F4861B8093A1
:1042600015010895109215010895809114016817A1
:1042700020F4861B80931401089510921401089570
:1042800080911301681720F4861B80931301089511
:1042900010921301089580911201681720F4861B73
:1042A00080931201089510921201089580911101D6
:1042B000681720F4861B8093110108951092110154
:1042C000089580911001681720F4861B80931001D7
:1042D00008951092100108950F931F938D3109F4E2
:1042E00071C008F045C0803109F485C008F58730F9
:1042F00009F46FC068F4863009F0ADC08091E30125
:10430000817F8E7F8093E30181E08093F301A4C0DD
:104310008B3009F49EC08E3009F09DC08091E3017E
:1043200082FB222720F991E0922790FB82F96CC052
:10433000863109F48EC060F4813109F08CC00E948E
:10434000E21690910D0181E0892780930D0181C0D3
:10435000893109F47EC08B3109F07DC08091E30181
:1043600081FB222720F991E0922790FB81F94CC034
:10437000853309F466C048F4873209F462C008F452
:104380004FC0893209F45DC066C0833438F48A3383
:1043900008F044C0883309F45CC05DC0833409F47C
:1043A00050C0883409F057C00E94E2160FEF13ED99
:1043B00020E3015010402040E1F700C000000E94BF
:1043C000041E47C00E94F6220E9449120E94460B1A
:1043D00040C09091E301892F8095817080FB90F916
:1043E00029F0966098609093E30136C0997F977F9B
:1043F0009093E3012EC08091E30183FB222720F9F3
:1044000091E0922790FB83F98093E301992309F1CE
:104410008091E30181608093E3011BC0895301C057
:104420008D5141E050E060E070E08A019B0104C0E2
:10443000000F111F221F331F8A95D2F7C901B8013F
:1044400004C061E070E080E090E00E94A21A0E9447
:10445000E21681E001C080E01F910F91089580E095
:10446000089580E008958E518A3030F4E82FF0E00E
:10447000E65DFE4F8081089580E00895CF93C82FB8
:104480008091F301813079F018F08230E9F186C033
:10449000E0910E01F0910F018081813169F082324B
:1044A00009F07EC009C0E0910E01F0910F018081FA
:1044B000813111F0823261F48C2F0E942F22811100
:1044C00004C08C2F0E946C211DC081E090E01AC0B6
:1044D0008C2F0E943122811114C0C43179F048F42C
:1044E000CB3079F0C03109F05FC082E08093F301F6
:1044F00008C0C93219F0C83321F056C01092F30138
:1045000053C081E0817052C0C93281F110F5C431CD
:1045100069F1A8F4C73009F045C08AE0809315011D
:1045200094E19093140193E090931301809312010E
:1045300088E08093110188E28093100133C082EEFD
:104540008C0F863078F58C2F0E9433228093F201F5
:1045500029C0CE34E9F020F4CB3421F56AE013C051
:10456000C13579F0C235F1F461E00DC08091F201FE
:10457000882319F01092F20115C081E08093F301B5
:1045800015C061E006C08091F2010E94A6200AC019
:104590006AE08091F2010E941C2104C01092F30194
:1045A00080E004C081E002C080E0ACCFCF910895EC
:1045B000E1E8F0E080818860808380818160808391
:1045C0008FB7F89493E09093890090ED90938800D2
:1045D0008FBF0895EFE6F0E08081826080830895C8
:1045E000EFE6F0E080818D7F80830895EFE6F0E0D4
:1045F000908182E08927808308951F920F920FB6E1
:104600000F9211242F933F934F935F936F937F9358
:104610008F939F93AF93BF93EF93FF938091F40198
:104620009091F50101969093F5018093F401811129
:1046300003C082E00E94460BE091F501E695E69505
:10464000F0E0E756FA4FE4918091F4018E1303C035
:1046500080E00E94460BFF91EF91BF91AF919F9137
:104660008F917F916F915F914F913F912F910F901B
:104670000FBE0F901F90189504D06894B1118DC093
:10468000089570D088F09F5790F0B92F9927B751AF
:10469000A0F0D1F0660F771F881F991F1AF0BA9506
:1046A000C9F712C0B13081F077D0B1E0089574C07D
:1046B000672F782F8827B85F39F0B93FCCF38695FC
:1046C00077956795B395D9F73EF490958095709559
:1046D00061957F4F8F4F9F4F0895E89409C097FBD6
:1046E0003EF490958095709561957F4F8F4F9F4FC9
:1046F0009923A9F0F92F96E9BB279395F69587950D
:1047000077956795B795F111F8CFFAF4BB0F11F4CF
:1047100060FF1BC06F5F7F4F8F4F9F4F16C0882376
:1047200011F096E911C0772321F09EE8872F762FAC
:1047300005C0662371F096E8862F70E060E02AF0ED
:104740009A95660F771F881FDAF7880F96958795D9
:1047500097F9089557FD9058440F551F59F05F3F42
:1047600071F04795880F97FB991F61F09F3F79F093
:1047700087950895121613061406551FF2CF469515
:10478000F1DF08C0161617061806991FF1CF869597
:104790007105610508940895E894BB27662777277B
:1047A000CB0197F908950BD078C069D028F06ED06E
:1047B00018F0952309F05AC05FC01124EECFCADF6C
:1047C000A0F3959FD1F3950F50E0551F629FF00124
:1047D000729FBB27F00DB11D639FAA27F00DB11D7D
:1047E000AA1F649F6627B00DA11D661F829F222706
:1047F000B00DA11D621F739FB00DA11D621F839F8D
:10480000A00D611D221F749F3327A00D611D231F62
:10481000849F600D211D822F762F6A2F11249F57B0
:1048200050408AF0E1F088234AF0EE0FFF1FBB1FD3
:10483000661F771F881F91505040A9F79E3F510572
:1048400070F014C0AACF5F3FECF3983EDCF386957E
:1048500077956795B795F795E7959F5FC1F7FE2B1D
:10486000880F911D9695879597F9089597F99F67F9
:1048700080E870E060E008959FEF80EC08950024E8
:104880000A941616170618060906089500240A94B5
:1048900012161306140605060895092E0394000C3B
:1048A00011F4882352F0BB0F40F4BF2B11F460FFCA
:1048B00004C06F5F7F4F8F4F9F4F089597FB072E68
:1048C00016F4009407D077FD09D00E94782407FCE5
:1048D00005D03EF4909581959F4F08957095619510
:1048E0007F4F0895EE0FFF1F0590F491E02D09947E
:1048F000AA1BBB1B51E107C0AA1FBB1FA617B70706
:1049000010F0A61BB70B881F991F5A95A9F7809521
:104910009095BC01CD010895F999FECF92BD81BD5E
:10492000F89A992780B50895A8E1B0E042E050E0F8
:104930000C94B424262FF999FECF92BD81BDF89A2C
:10494000019700B4021639F01FBA20BD0FB6F894D3
:10495000FA9AF99A0FBE08950196272F0E949B2478
:104960000C949A24DC01CB01FC01F999FECF06C01E
:10497000F2BDE1BDF89A319600B40D92415050401D
:08498000B8F70895F894FFCF89
:104988000220480BD60BB30B7F0B4B0B0101D00158
:1049980028080A03140A404D363959050C05D6046F
:1049A8009D043004490462047B04010203040506E3
:0449B80007080900E3
:00000001FF
